:020000040800F2
:1000000000060220010200080302000803020008A3
:1000100003020008030200080302000803020008AC
:10002000030200080302000803020008A1370008C9
:10003000030200080302000803020008030200088C
:10004000030200080302000803020008030200087C
:100050000302000803020008453A00086D3A000850
:10006000953A0008BD3A0008E53A00080302000886
:10007000030200080302000803020008030200084C
:10008000030200080302000803020008030200083C
:100090000302000803020008030200080D3B0008E9
:1000A000030200080302000803020008030200081C
:1000B000F53B0008030200080302000803020008E1
:1000C00003020008030200080302000803020008FC
:1000D00003020008030200080302000803020008EC
:1000E000713B000803020008030200080302000835
:1000F00003020008030200080302000803020008CC
:1001000003020008030200080302000803020008BB
:1001100003020008030200080302000803020008AB
:10012000030200080302000803020008030200089B
:10013000030200080302000803020008030200088B
:10014000030200080302000803020008192F000838
:10015000030200080302000803020008030200086B
:10016000030200080302000803020008030200085B
:10017000030200080302000803020008030200084B
:100180000302000803020008E13B00080302000824
:10019000030200080302000803020008030200082B
:1001A000030200080302000803020008030200081B
:1001B000030200080302000803020008030200080B
:1001C00003020008030200080302000803020008FB
:1001D00003020008030200080302000803020008EB
:1001E00003020008030200080302000803020008DB
:1001F00003020008030200080302000803020008CB
:1002000002E000F000F8FEE772B6374880F3088895
:10021000364880F3098836483649086040F20000C5
:10022000CCF200004EF63471CEF200010860BFF34C
:100230004F8FBFF36F8F40F20000C0F2F0004EF618
:100240008851CEF200010860BFF34F8FBFF36F8F6C
:100250004FF00000E1EE100A4EF63C71CEF20001C4
:100260000860062080F31488BFF36F8F02F0B2FAA3
:1002700003F028FA4FF055301F491B4A91423CBF0A
:1002800041F8040BFAE71D49184A91423CBF41F876
:10029000040BFAE71A491B4A1B4B9A423EBF51F81E
:1002A000040B42F8040BF8E700201849184A914261
:1002B0003CBF41F8040BFAE702F0CAFA03F062FA15
:1002C000144C154DAC4203DA54F8041B8847F9E787
:1002D00000F042F8114C124DAC4203DA54F8041B02
:1002E0008847F9E702F0B2BA000602200022022095
:1002F0000000000808ED00E00000022000060220D7
:1003000010400008002202206422022068220220FD
:100310003835022000020008000200080002000830
:10032000000200082DE9F04F2DED108AC1F80CD025
:10033000D0F80CD0BDEC108ABDE8F08F002383F319
:1003400011882846A047002001F0F2FDFEE701F0E9
:1003500081FD00DFFEE7000038B500F0B7FB02F0DA
:10036000F9F9054602F02CFA0446D0B90F4B9D422C
:1003700019D001339D4241F2883512BF0446002551
:100380000124002002F0F0F90CB100F077F800F041
:1003900071FD00F017FC284600F0FAF800F06EF846
:1003A000F9E70025EDE70546EBE700BF010007B0E0
:1003B00008B500F0D3FBA0F120035842584108BD16
:1003C00007B541F21203022101A8ADF8043000F094
:1003D000E3FB03B05DF804FB38B5302383F31188E9
:1003E000174803680BB101F06FFE0023154A4FF464
:1003F0007A71134801F05EFE002383F31188124CDA
:10040000236813B12368013B2360636813B16368F9
:10041000013B63600D4D2B7833B963687BB90220D3
:1004200000F0A2FC322363602B78032B07D16368B2
:100430002BB9022000F098FC4FF47A73636038BD4A
:1004400068220220D903000888230220802202208B
:10045000084B187003280CD8DFE800F008050208E4
:10046000022000F077BC022000F06ABC024B0022A0
:100470005A6070478022022088230220F8B53F4B43
:100480003F4A1C461968013177D004339342F9D1B1
:100490006268A24271D33B4B9B6803F1006303F592
:1004A000C0339A4269D2002000F0A6FB0220FFF779
:1004B000CFFF354B00211A6C19641A6E19661A6E3B
:1004C0005A6C59645A6E59665A6E5A6942F08002E3
:1004D0005A615A6922F080025A615A691A6942F0D7
:1004E00000521A611A6922F000521A611B6972B631
:1004F0004FF0E023C3F8084DD4E90004BFF34F8F59
:10050000BFF36F8F214AC2F88410BFF34F8F536936
:1005100023F480335361BFF34F8FD2F8803043F61A
:10052000E076C3F3C905C3F34E335B0103EA060C5F
:1005300029464CEA81770139C2F87472F9D2203B1E
:1005400013F1200FF2D1BFF34F8FBFF36F8FBFF3C3
:100550004F8FBFF36F8F536923F400335361002330
:10056000C2F85032BFF34F8FBFF36F8F302383F346
:100570001188854680F308882047F8BD008001086F
:1005800020800108002202200038024000ED00E037
:100590002DE9F04F93B0B44B2022FF2100900AA820
:1005A0009D6800F011FCB14A1378A3B90121B0484D
:1005B00011700360302383F3118803680BB101F0DD
:1005C00083FD0023AB4A4FF47A71A94801F072FD14
:1005D000002383F31188009B13B1A74B009A1A6084
:1005E000A64A1378032B03D000231370A24A53604A
:1005F0004FF0000A009CD3465646D146012000F039
:10060000A9FB24B19C4B1B68002B00F02682002024
:1006100000F0A4FA0390039B002BF2DB012000F012
:100620008FFB039B213B1F2BE8D801A252F823F03C
:10063000B1060008D90600086D070008FD0500088E
:10064000FD050008FD050008FF070008CF090008A8
:10065000E90800084B090008730900089909000817
:10066000FD050008AB090008FD0500081D0A00088B
:1006700051070008FD050008610A0008BD060008D2
:1006800051070008FD0500084B090008FD0500089A
:10069000FD050008FD050008FD050008FD05000832
:1006A000FD050008FD050008FD0500086D070008B0
:1006B0000220FFF77DFE002840F0F981009B022117
:1006C00005A8BAF1000F08BF1C4641F21233ADF87D
:1006D000143000F061FA91E74FF47A7000F03EFABE
:1006E000071EEBDB0220FFF763FE0028E6D0013F88
:1006F000052F00F2DE81DFE807F0030A0D10133644
:100700000523042105A8059300F046FA17E004210B
:100710005548F9E704215A48F6E704215948F3E718
:100720004FF01C08404608F1040800F067FA042165
:10073000059005A800F030FAB8F12C0FF2D1012095
:100740004FF0000900FA07F747EA0B0B5FFA8BFB43
:1007500000F086FB26B10BF00B030B2B08BF002427
:10076000FFF72EFE4AE704214748CDE7002EA5D02B
:100770000BF00B030B2BA1D10220FFF719FE07464C
:1007800000289BD00120002600F036FA0220FFF757
:100790005FFE1FFA86F8404600F03EFA0446B0B10C
:1007A000039940460136A1F140025142514100F007
:1007B00043FA0028EDD1BA46044641F21213022151
:1007C00005A83E46ADF8143000F0E6F916E72546D8
:1007D0000120FFF73DFE244B9B68AB4207D928461A
:1007E00000F00CFA013040F067810435F3E7002592
:1007F000224BBA463E461D701F4B5D60A8E7002E97
:100800003FF45CAF0BF00B030B2B7FF457AF0220D0
:10081000FFF71EFE322000F0A1F9B0F10008FFF64C
:100820004DAF18F003077FF449AF0F4A08EB0503FB
:10083000926893423FF642AFB8F5807F3FF73EAFF4
:10084000124BB845019323DD4FF47A7000F086F91E
:100850000390039A002AFFF631AF039A0137019BF8
:1008600003F8012BEDE700BF0022022084230220C1
:1008700068220220D9030008882302208022022057
:1008800004220220082202200C22022084220220BC
:10089000C820FFF78DFD074600283FF40FAF1F2D3E
:1008A00011D8C5F120020AAB25F003008449424566
:1008B000184428BF4246019200F060FA019AFF21D5
:1008C0007F4800F081FA4FEAA803C8F387027C4909
:1008D0002846019300F080FA064600283FF46DAFE9
:1008E000019B05EB830533E70220FFF761FD00283C
:1008F0003FF4E4AE00F0CCF900283FF4DFAE00276F
:10090000B846704B9B68BB4218D91F2F11D80A9B61
:1009100001330ED027F0030312AA134453F8203CEE
:1009200005934046042205A9043700F003FB8046E6
:10093000E7E7384600F062F90590F2E7CDF8148059
:10094000042105A800F028F902E70023642104A887
:10095000049300F017F900287FF4B0AE0220FFF7EF
:1009600027FD00283FF4AAAE049800F079F905901D
:10097000E6E70023642104A8049300F003F90028AB
:100980007FF49CAE0220FFF713FD00283FF496AEE3
:10099000049800F075F9EAE70220FFF709FD002846
:1009A0003FF48CAE00F084F9E1E70220FFF700FD90
:1009B00000283FF483AE05A9142000F07FF9074614
:1009C0000421049004A800F0E7F83946B9E7322082
:1009D00000F0C4F8071EFFF671AEBB077FF46EAEE1
:1009E000384A07EB0903926893423FF667AE02204C
:1009F000FFF7DEFC00283FF461AE27F003074F4409
:100A0000B9453FF4A5AE484609F1040900F0F6F8EF
:100A10000421059005A800F0BFF8F1E74FF47A70C3
:100A2000FFF7C6FC00283FF449AE00F031F900287A
:100A300044D00A9B01330BD008220AA9002000F001
:100A4000CBF900283AD02022FF210AA800F0BCF9F7
:100A5000FFF7B6FC1C4801F071FA13B0BDE8F08F47
:100A6000002E3FF42BAE0BF00B030B2B7FF426AEC6
:100A70000023642105A8059300F084F807460028A8
:100A80007FF41CAE0220FFF793FC804600283FF461
:100A900015AEFFF795FC41F2883001F04FFA05984A
:100AA00000F026FA46463C4600F0DAF9A6E506468E
:100AB0004EE64FF0000901E6BA467EE637467CE690
:100AC0008422022000220220A0860100704700003C
:100AD0002DE9F84F4FF47A7306460D46002402FBC9
:100AE00003F7DFF85080DFF8509098F900305FFA94
:100AF00084FA5A1C01D0A34212D159F824002A4684
:100B000031460368D3F820B03B46D847854207D129
:100B1000074B012083F800A0BDE8F88F0124E4E72B
:100B2000002CFBD04FF4FA7001F008FA0020F3E734
:100B3000D4230220102202201422022070B5044681
:100B40004FF47A76412C254628BF412506FB05F057
:100B500001F0F4F9641BF5D170BD0000002307B566
:100B6000024601210DF107008DF80730FFF7B0FFB5
:100B700020B19DF8070003B05DF804FB4FF0FF3093
:100B8000F9E700000A46042108B5FFF7A1FF80F04D
:100B90000100C0B2404208BD074B0A4630B4197884
:100BA000064B53F82140014623682046DD69044B7B
:100BB000AC4630BC604700BFD42302201422022080
:100BC000A086010070B50A4E00240A4D01F0C8FC51
:100BD000308028683388834208D901F0BBFC2B6839
:100BE00004440133B4F5C03F2B60F2D370BD00BFA5
:100BF000D62302209023022001F060BD00F10060A6
:100C000000F5C0300068704700F10060920000F508
:100C1000C03001F0EBBC0000054B1A68054B1B8887
:100C20009B1A834202D9104401F094BC0020704703
:100C300090230220D623022038B50446074D29B15F
:100C400028682044BDE8384001F0A4BC286820444E
:100C500001F088FC0028F3D038BD00BF90230220AB
:100C600010F0030309D1B0F5846F04D200F10050F5
:100C7000A0F571200368184670470023FBE70000C9
:100C800000F10050A0F57120D0F82004704700005A
:100C9000064991F8243033B100230822086A81F80C
:100CA0002430FFF7B1BF0120704700BF942302201A
:100CB000014B1868704700BF002004E01E4B01384C
:100CC000F0B51D680A1803231C482E0CC5F30B044D
:100CD00035460788A7420BD144680B46013C934236
:100CE00018461BD214F9010F48B103F8010BF6E7BF
:100CF000013B00F10800ECD191420ED20B461846A0
:100D00002C24B6F5805F00F8014B0AD1824202D94B
:100D10004122981C5A70401AF0BD0846B6F5805F13
:100D2000F9D041F201039D42F5D18242F3D95A2311
:100D300000F8013BEFE700BF002004E01C22022086
:100D4000022803D1024B4FF080629A61704700BFC6
:100D5000000C0240022803D1024B4FF480629A61DA
:100D6000704700BF000C0240022804D1024A5369B8
:100D700083F4806353617047000C0240002310B578
:100D8000934203D0CC5CC4540133F9E710BD00009A
:100D9000013810B510F9013F3BB191F900409C4278
:100DA00003D11AB10131013AF4E71AB191F90020E7
:100DB000981A10BD1046FCE703460246D01A12F9F5
:100DC000011B0029FAD1704702440346934202D026
:100DD00003F8011BFAE770472DE9F8431F4D14464D
:100DE0000746884695F8242052BBDFF870909CB3E4
:100DF00095F824302BB92022FF2148462F62FFF7B7
:100E0000E3FF95F824004146C0F1080205EB80009D
:100E1000A24228BF2246D6B29200FFF7AFFF95F854
:100E20002430A41B17441E449044E4B2F6B2082EAA
:100E300085F82460DBD1FFF72BFF0028D7D108E02D
:100E40002B6A03EB82038342CFD0FFF721FF0028F8
:100E5000CBD10020BDE8F8830120FBE794230220DA
:100E6000024B1A78024B1A70704700BFD42302203D
:100E70001022022038B5194C194D204600F0BCFB59
:100E80002946204600F0E4FB2D684FF47A70EA6EA4
:100E9000D2F8043843F00203C2F80438FFF74EFEDC
:100EA0001049284600F0DCFCEA6E0F4DD2F80438F9
:100EB000286823F002030D49A042C2F804384FF419
:100EC000E1330B6001D000F0F7FA6868A04204D06B
:100ED0000649BDE8384000F0EFBA38BDB828022016
:100EE000BC3D0008C43D000814220220BC2302209F
:100EF0000C4B70B50C4D04461E780C4B55F8262053
:100F00009A420DD00A4B002118221846FFF75CFFC9
:100F10000460014655F82600BDE8704000F0CCBAE8
:100F200070BD00BFD423022014220220B828022062
:100F3000BC23022030B50A44084D91420DD011F86F
:100F4000013B5840082340F30004013B2C4013F0C0
:100F5000FF0384EA5000F6D1EFE730BD2083B8EDFF
:100F6000026843681143016003B1184770470000ED
:100F7000024A136843F0C0031360704700780040D2
:100F800013B50E4C204600F08BFA04F11400002338
:100F90004FF480720A49009400F048F9094B4FF46D
:100FA0008072094904F13800009400F0C1F9074A41
:100FB000074BC4E9172302B010BD00BFD82302209D
:100FC00044240220710F00084425022000780040CC
:100FD00080F93703037C30B5214C002918BF0C463B
:100FE000012B0CD11F4B984209D11F4B1A6C42F0B8
:100FF00080421A641A6E42F080421A661B6E2268A2
:10100000036EC16D03EB52038466B3FBF2F36268B7
:10101000150442BF23F0070503F0070343EA450325
:10102000CB60A36843F040034B60E36843F00103E7
:101030008B6042F4967343F001030B604FF0FF3373
:101040000B62510505D512F0102205D0B2F1805F78
:1010500004D080F8643030BD7F23FAE73F23F8E7FF
:10106000D03C0008D8230220003802402DE9F04788
:10107000C66D05463768F469210734621AD014F04A
:10108000080118BF4FF48071E20748BF41F020010A
:10109000A3074FF0300348BF41F04001600748BF4D
:1010A00041F0800183F31188281DFFF759FF0023C9
:1010B00083F31188E2050AD5302383F311884FF4B6
:1010C0008061281DFFF74CFF002383F311884FF048
:1010D00030094FF0000A14F0200838D13B0616D52D
:1010E0004FF0300905F1380A200610D589F3118830
:1010F000504600F051F9002836DA0821281DFFF784
:101100002FFF27F080033360002383F311887906D3
:1011100014D5620612D5302383F31188D5E9132341
:101120009A4208D12B6C33B127F040071021281DBB
:10113000FFF716FF3760002383F31188E30618D505
:10114000AA6E1369ABB15069BDE8F047184789F33F
:101150001188736A284695F86410194000F0BAF9AE
:101160008AF31188F469B6E7B06288F31188F469EC
:10117000BAE7BDE8F0870000F8B515468268044676
:101180000B46AA4200D28568A1692669761AB54243
:101190000BD218462A46FFF7F1FDA3692B44A36141
:1011A0002846A3685B1BA360F8BD0CD9AF1B18468B
:1011B0003246FFF7E3FD3A46E1683044FFF7DEFDD3
:1011C000E3683B44EBE718462A46FFF7D7FDE368A0
:1011D000E5E7000083689342F7B50446154600D260
:1011E0008568D4E90460361AB5420BD22A46FFF767
:1011F000C5FD63692B4463612846A3685B1BA3603C
:1012000003B0F0BD0DD93246AF1B0191FFF7B6FD1B
:1012100001993A46E0683144FFF7B0FDE3683B448A
:10122000E9E72A46FFF7AAFDE368E4E710B50A44B8
:101230000024C361029B8460C16002610362C0E953
:101240000000C0E9051110BD08B5D0E90532934290
:1012500001D1826882B98268013282605A1C42617F
:1012600019700021D0E904329A4224BFC368436157
:1012700000F080FE002008BD4FF0FF30FBE70000CB
:1012800070B5302304460E4683F31188A568A5B1D6
:10129000A368A269013BA360531CA361157822696E
:1012A000934224BFE368A361E3690BB120469847EA
:1012B000002383F31188284607E03146204600F0DA
:1012C00049FE0028E2DA85F3118870BD2DE9F74F59
:1012D00004460E4617469846D0F81C904FF0300A48
:1012E0008AF311884FF0000B154665B12A46314646
:1012F0002046FFF741FF034660B94146204600F013
:1013000029FE0028F1D0002383F31188781B03B055
:10131000BDE8F08FB9F1000F03D001902046C84717
:10132000019B8BF31188ED1A1E448AF31188DCE7C8
:10133000C160C361009B82600362C0E90511114472
:10134000C0E9000001617047F8B504460D46164635
:10135000302383F31188A768A7B1A368013BA3607A
:1013600063695A1C62611D70D4E904329A4224BF39
:10137000E3686361E3690BB120469847002080F37E
:10138000118807E03146204600F0E4FD0028E2DA4B
:1013900087F31188F8BD0000D0E9052310B59A4203
:1013A00001D182687AB982680021013282605A1CB8
:1013B00082611C7803699A4224BFC368836100F08C
:1013C000D9FD204610BD4FF0FF30FBE72DE9F74F68
:1013D00004460E4617469846D0F81C904FF0300A47
:1013E0008AF311884FF0000B154665B12A46314645
:1013F0002046FFF7EFFE034660B94146204600F065
:10140000A9FD0028F1D0002383F31188781B03B0D5
:10141000BDE8F08FB9F1000F03D001902046C84716
:10142000019B8BF31188ED1A1E448AF31188DCE7C7
:10143000026843681143016003B118477047000018
:101440001430FFF743BF00004FF0FF331430FFF7B5
:101450003DBF00003830FFF7B9BF00004FF0FF3349
:101460003830FFF7B3BF00001430FFF709BF0000AA
:101470004FF0FF311430FFF703BF00003830FFF7A3
:1014800063BF00004FF0FF323830FFF75DBF000050
:10149000012914BF6FF0130000207047FFF770BDE3
:1014A000044B036000234360C0E90233012303744B
:1014B000704700BFE83C000810B53023044683F3B2
:1014C0001188FFF787FD02230020237480F3118821
:1014D00010BD000038B5C36904460D461BB9042190
:1014E0000844FFF7A5FF294604F11400FFF7ACFEFE
:1014F000002806DA201D4FF40061BDE83840FFF7F0
:1015000097BF38BD026843681143016003B11847B3
:101510007047000013B5446BD4F8A4381A681178EA
:10152000042915D1217C022912D1197901231289AC
:101530008B4013420CD101A904F14C0001F07EFF55
:10154000D4F8A4480246019B2179206800F0D6F91E
:1015500002B010BD143001F001BF00004FF0FF33A6
:10156000143001F0FBBE00004C3001F0D3BF00008E
:101570004FF0FF334C3001F0CDBF0000143001F0CC
:10158000CFBE00004FF0FF31143001F0C9BE0000A3
:101590004C3001F09FBF00004FF0FF324C3001F0A3
:1015A00099BF000000207047D0F8A4381A6810B521
:1015B00011780446042917D1017C022914D15979E4
:1015C000012352898B4013420ED1143001F062FE88
:1015D000024648B1D4F8A4484FF48073617920687A
:1015E000BDE8104000F078B910BD0000406BFFF777
:1015F000DBBF0000704700007FB5124B01250426B9
:10160000044603600023057400F184024360294608
:10161000C0E902330C4B0290143001934FF48073F5
:10162000009601F013FE094B04F29442294604F19E
:101630004C000294CDE900634FF4807301F0DAFEB0
:1016400004B070BD103D0008ED1500081515000828
:101650000B68302282F311880A7903EB8202106250
:101660004A790D3243F822008A7912B103EB8203E2
:1016700018620223C0F8A4180374002080F31188B4
:101680007047000038B5037F044613B190F854301A
:10169000ABB90125201D0221FFF734FF04F114002E
:1016A0006FF00101257700F071FC04F14C0084F823
:1016B00054506FF00101BDE8384000F067BC38BD00
:1016C00010B5012104460430FFF71CFF00232377E7
:1016D00084F8543010BD000038B50446002514309D
:1016E00001F0CCFD04F14C00257701F09BFE201D9C
:1016F00084F854500121FFF705FF2046BDE838402B
:10170000FFF752BF90F85C3003F06003202B06D146
:1017100090F85D200023212A03D81F2A06D8002034
:101720007047222AFBD1C0E9143303E0034A026563
:101730000722426583650120704700BF34220220E2
:10174000D0F8A43837B51A680446117804291AD19C
:10175000017C022917D11979012312898B40134288
:1017600011D100F14C05284601F01CFF58B101A928
:10177000284601F063FED4F8A4480246019B217973
:10178000206800F0BBF803B030BD000000EB81031F
:10179000F0B51E6A85B004460D46FEB1302383F3D2
:1017A000118804EB8507301D0821FFF7ABFEFB68AD
:1017B00006F14C005B691B681BB1019001F04CFE07
:1017C000019803A901F03AFE024648B1039B29465D
:1017D000204600F093F8002383F3118805B0F0BD94
:1017E000FB685A691268002AF5D01B8A013B134036
:1017F000F1D104F15C02EAE70D3138B550F821402F
:10180000DCB1302383F31188D4F8A428136852790B
:1018100003EB8203DB689B695D6845B104216018B6
:10182000FFF770FE294604F1140001F03DFD20464B
:10183000FFF7BAFE002383F3118838BD704700001C
:1018400001F08AB801232822002110B5044600F8CF
:10185000243BFFF7B9FA0023C4E9013310BD0000AF
:1018600038B50446302383F3118800254160C0E970
:101870000355C0E90555C0E9075501F07DF802237D
:10188000237085F31188284638BD000070B500EB41
:101890008103054650690E461446DA6018B11022DD
:1018A0000021FFF791FAA06918B110220021FFF77B
:1018B0008BFA31462846BDE8704001F027B9000098
:1018C000826802F0011282600022C0E90422C0E9AD
:1018D0000622026201F0A6B9F0B4012500EB8104F2
:1018E00047898D40E4683D43A46945812360002316
:1018F000A2606360F0BC01F0C1B90000F0B4012542
:1019000000EB810407898D40E4683D4364690581EB
:1019100023600023A2606360F0BC01F03BBA0000CA
:1019200070B502230025044603704566056280F801
:101930004C50C0E90255C0E90455C0E9065501F014
:1019400081F863681B6823B129462046BDE87040D2
:10195000184770BD0378052B10B504460AD080F8EF
:1019600068300523037043681B680BB10421984756
:101970000023A36010BD00000178052906D190F86E
:101980006820436802701B6803B118477047000065
:1019900070B590F84C30044613B1002380F84C30F9
:1019A00004F15C02204601F05FF963689B68B3B9FB
:1019B00094F85C3013F0600535D00021204601F02A
:1019C00011FC0021204601F003FC63681B6813B181
:1019D000062120469847062384F84C3070BD2046E7
:1019E00098470028E4D0B4F86230626D9A4288BF0C
:1019F000636594F95C30656D002B4FF0300380F225
:101A00000381002D00F0F280092284F84C2083F33A
:101A1000118800212046D4E91423FFF76FFF00232B
:101A200083F31188DAE794F85D2003F07F0343EA3B
:101A3000022340F20232934200F0C58021D8B3F570
:101A4000807F48D00DD8012B3FD0022B00F093802F
:101A5000002BB2D104F16402226502226265A36503
:101A6000C1E7B3F5817F00F09B80B3F5407FA4D13F
:101A700094F85E30012BA0D1B4F8643043F0020337
:101A800032E0B3F5006F4DD017D8B3F5A06F31D069
:101A9000A3F5C063012B90D86368204694F85E20BC
:101AA0005E6894F85F10B4F86030B047002884D0C6
:101AB00043682365036863651AE0B3F5106F36D099
:101AC00040F6024293427FF478AF5C4B23650223D9
:101AD00063650023C3E794F85E30012B7FF46DAF9C
:101AE000B4F8643023F00203A4F86430C4E9145558
:101AF000A56578E7B4F85C30B3F5A06F0ED194F823
:101B00005E30204684F8663000F0F4FF63681B689E
:101B100013B1012120469847032323700023C4E911
:101B200014339CE704F1670323650123C3E723789B
:101B3000042B10D1302383F311882046FFF7C0FE19
:101B400085F311880321636884F8675021701B684E
:101B50000BB12046984794F85E30002BDED084F815
:101B600067300423237063681B68002BD6D00221E2
:101B700020469847D2E794F8603020461D0603F0CF
:101B80000F010AD501F062F8012804D002287FF481
:101B900014AF2B4B9AE72B4B98E701F049F8F3E78A
:101BA00094F85E30002B7FF408AF94F8603013F0A7
:101BB0000F01B3D01A06204602D501F027FBADE78E
:101BC00001F01AFBAAE794F85E30002B7FF4F5AE23
:101BD00094F8603013F00F01A0D01B06204602D508
:101BE00001F000FB9AE701F0F3FA97E7142284F87A
:101BF0004C2083F311882B462A4629462046FFF7BE
:101C00006BFE85F31188E9E65DB1152284F84C205E
:101C100083F3118800212046D4E91423FFF75CFEEA
:101C2000FDE60B2284F84C2083F311882B462A46CC
:101C300029462046FFF762FEE3E700BF403D00086B
:101C4000383D00083C3D000838B590F84C3004465B
:101C5000002B3ED0063BDAB20F2A34D80F2B32D8F5
:101C6000DFE803F03731310822323131313131319F
:101C700031313737456DB0F862309D4214D2C368B8
:101C80001B8AB5FBF3F203FB12556DB9302383F3C6
:101C900011882B462A462946FFF730FE85F3118826
:101CA0000A2384F84C300EE0142384F84C3030239F
:101CB00083F31188002320461A461946FFF70CFECD
:101CC000002383F3118838BD836D03B19847002347
:101CD000E7E70021204601F085FA0021204601F0C7
:101CE00077FA63681B6813B10621204698470623DC
:101CF000D7E7000010B590F84C300446142B29D0DB
:101D000017D8062B05D001D81BB110BD093B022BFB
:101D1000FBD80021204601F065FA0021204601F0A1
:101D200057FA63681B6813B10621204698470623BB
:101D300019E0152BE9D10B2380F84C30302383F3C5
:101D4000118800231A461946FFF7D8FD002383F3B4
:101D50001188DAE7C3689B695B68002BD5D1836D76
:101D600003B19847002384F84C30CEE70023826803
:101D7000037503691B6899689142FBD25A68036036
:101D800042601060586070470023826803750369E1
:101D90001B6899689142FBD85A68036042601060E2
:101DA0005860704708B50846302383F311880B7DCF
:101DB000032B05D0042B0DD02BB983F3118808BD5C
:101DC0008B6900221A604FF0FF338361FFF7CEFF6B
:101DD0000023F2E7D1E9003213605A60F3E7000014
:101DE000FFF7C4BF054BD9680875186802685360CF
:101DF0001A600122D8600275FEF794BA48260220C4
:101E00000C4B30B5DD684B1C87B004460FD02B4619
:101E1000094A684600F04EF92046FFF7E3FF009BB1
:101E200013B1684600F050F9A86907B030BDFFF75C
:101E3000D9FFF9E748260220A51D0008044B1A68BF
:101E4000DB6890689B68984294BF0020012070472F
:101E500048260220084B10B51C68D86822685360D9
:101E60001A600122DC602275FFF78EFF01462046D2
:101E7000BDE81040FEF756BA4826022038B5074C98
:101E800001230025064907482370656001F0C2FB65
:101E90000223237085F3118838BD00BFB0280220CB
:101EA000483D00084826022000F044B9034A516822
:101EB00053685B1A9842FBD8704700BF001000E0DF
:101EC0008B600223086108468B8270478368A3F108
:101ED000840243F8142C026943F8442C426943F805
:101EE000402C094A43F8242CC268A3F1200043F88F
:101EF000182C022203F80C2C002203F80B2C034AA6
:101F000043F8102C704700BF3D030008482602200C
:101F100008B5FFF7DBFFBDE80840FFF761BF000031
:101F2000024BDB6898610F20FFF75CBF4826022058
:101F3000302383F31188FFF7F3BF000008B5014693
:101F4000302383F311880820FFF75AFF002383F31F
:101F5000118808BD064BDB6839B1426818605A60C9
:101F6000136043600420FFF74BBF4FF0FF30704712
:101F7000482602200368984206D01A680260506022
:101F800018469961FFF72CBF7047000038B504462A
:101F90000D462068844200D138BD036823605C6030
:101FA0008561FFF71DFFF4E7036810B59C68A24246
:101FB0000CD85C688A600B604C602160596099683D
:101FC0008A1A9A604FF0FF33836010BD121B1B68A2
:101FD000ECE700000A2938BF0A2170B504460D4617
:101FE0000A26601901F010FB01F0FCFA041BA5425F
:101FF00003D8751C04462E46F3E70A2E04D90120A7
:10200000BDE8704001F046BB70BD0000F8B5144B50
:102010000D460A2A4FF00A07D96103F110018260C8
:1020200038BF0A224160196914460160486018618E
:10203000A81801F0DBFA01F0D5FA431B0646A342CB
:1020400006D37C1C28192746354601F0DDFAF2E755
:102050000A2F04D90120BDE8F84001F01BBBF8BDF0
:1020600048260220F8B506460D4601F0BBFA0F4A95
:10207000134653F8107F9F4206D12A460146304648
:10208000BDE8F840FFF7C2BFD169BB68441A2C19FC
:1020900028BF2C46A34202D92946FFF79BFF2246C0
:1020A00031460348BDE8F840FFF77EBF48260220CE
:1020B00058260220C0E90323002310B45DF8044B26
:1020C0004361FFF7CFBF000010B5194C2369984258
:1020D0000DD08168D0E9003213605A609A680A44D2
:1020E0009A60002303604FF0FF33A36110BD0268C4
:1020F000234643F8102F53600022026022699A425F
:1021000003D1BDE8104001F079BA936881680B44AF
:10211000936001F067FA2269E1699268441AA24269
:10212000E4D91144BDE81040091AFFF753BF00BFBE
:10213000482602202DE9F047DFF8BC8008F110079F
:102140002C4ED8F8105001F04DFAD8F81C40AA686F
:10215000031B9A423ED814444FF00009D5E90032DF
:10216000C8F81C4013605A60C5F80090D8F81030C9
:10217000B34201D101F042FA89F31188D5E9033164
:1021800028469847302383F311886B69002BD8D0F9
:1021900001F028FA6A69A0EB040982464A450DD28B
:1021A000022001F077FA0022D8F81030B34208D1AB
:1021B00051462846BDE8F047FFF728BF121A2244CF
:1021C000F2E712EB09092946384638BF4A46FFF7BD
:1021D000EBFEB5E7D8F81030B34208D01444C8F885
:1021E0001C00211AA960BDE8F047FFF7F3BEBDE867
:1021F000F08700BF582602204826022000207047A2
:10220000FEE70000704700004FF0FF30704700000D
:1022100002290CD0032904D00129074818BF002047
:102220007047032A05D8054800EBC20070470448F0
:1022300070470020704700BF203E00084422022063
:10224000D43D000870B59AB005460846144601A969
:1022500000F0C2F801A8FEF7AFFD431C0022C6B291
:102260005B001046C5E9003423700323023404F8F0
:10227000013C01ABD1B202348E4201D81AB070BD1C
:1022800013F8011B013204F8010C04F8021CF1E7F9
:1022900008B5302383F311880348FFF751FA002370
:1022A00083F3118808BD00BFB828022090F85C3085
:1022B00003F01F02012A07D190F85D200B2A03D1F9
:1022C0000023C0E9143315E003F06003202B08D18C
:1022D000B0F860302BB990F85D20212A03D81F2A6E
:1022E00004D8FFF70FBA222AEBD0FAE7034A0265B7
:1022F0000722426583650120704700BF3B22022010
:1023000007B5052917D8DFE801F0191603191920B8
:10231000302383F31188104A01210190FFF7B6FAA8
:10232000019802210D4AFFF7B1FA0D48FFF7D4F9E1
:10233000002383F3118803B05DF804FB302383F39B
:1023400011880748FFF79EF9F2E7302383F31188DD
:102350000348FFF7B5F9EBE7743D0008983D000826
:10236000B828022038B50C4D0C4C2A460C4904F113
:102370000800FFF767FF05F1CA0204F110000949E0
:10238000FFF760FF05F5CA7204F118000649BDE8C1
:102390003840FFF757BF00BF90310220442202208F
:1023A000543D00085E3D0008693D000870B50446D4
:1023B00008460D46FEF700FDC6B2204601340378FC
:1023C0000BB9184670BD32462946FEF7E1FC0028DD
:1023D000F3D10120F6E700002DE9F04705460C4651
:1023E000FEF7EAFC2C49C6B22846FFF7DFFF08B12A
:1023F0000C36F6B229492846FFF7D8FF08B1103647
:10240000F6B2632E0BD8DFF89080DFF89090244F5F
:10241000DFF898A02E7846B92670BDE8F0872946E7
:102420002046BDE8F04701F035BC252E30D107220B
:1024300041462846FEF7ACFC80B91A4B224603F110
:10244000100153F8040B8B4242F8040BF9D11988A0
:1024500007359B78133411809370DBE708224946D7
:102460002846FEF795FC98B9A21C0F4B197802324A
:102470000909C95D02F8041C13F8011B01F00F01E2
:102480005345C95D02F8031CF0D118340835C1E783
:10249000013504F8016BBDE7403E0008693D0008C6
:1024A0005C3E0008483E000820F4F01F2CF4F01FAA
:1024B000BFF34F8F024AD368DB03FCD4704700BFE1
:1024C000003C024008B5074B1B7853B9FFF7F0FFFB
:1024D000054B1A69002A04DA044A5A6002F188326C
:1024E0005A6008BDEE330220003C024023016745DC
:1024F00008B5054B1B7833B9FFF7DAFF034A1369B8
:1025000043F00043136108BDEE330220003C02405B
:102510000B28F0B516D80C4C0C4923787BB90E4625
:102520000B4D0C234FF00062013B55F8047B46F83D
:10253000042B13F0FF033A44F6D10123237051F822
:102540002000F0BD0020FCE720340220F033022000
:10255000703E0008014B53F820007047703E0008A1
:102560000C2070470B2810B5044601D9002010BD7F
:10257000FFF7CEFF064B53F824301844C21A0BB9AC
:102580000120F4E712680132F0D1043BF6E700BF06
:10259000703E00080B2810B5044621D8FFF788FFCD
:1025A000FFF790FF0F4AF323D360C300DBB243F47D
:1025B000007343F002031361136943F48033136122
:1025C000FFF776FFFFF7A4FF074B53F8241000F046
:1025D000D9F82046FFF78CFFBDE81040FFF7C2BFD7
:1025E000002010BD003C0240703E0008F8B512F01B
:1025F0000103144642D18218B2F1026F57D82D4B15
:102600001B6813F0010352D0FFF75CFF2A4DF32340
:1026100040F20127EB60FFF74BFF032C15D824F0A5
:102620000104401A40F201176618234CB14200EB36
:102630000105236924D123F0010301202361FFF761
:1026400057FFF8BD043C0430E7E78307E7D12B6967
:1026500023F440732B612B693B432B6151F8046BCE
:102660000660BFF34F8FFFF723FF03689E42E9D058
:102670002B6923F001032B61FFF73AFF0020E0E70D
:1026800023F44073236123693B4323610B882B8030
:10269000BFF34F8FFFF70CFF2D88ADB231F8023B2F
:1026A000AB42C3D0236923F001032361E4E718465A
:1026B000C7E700BF00380240003C0240084908B5A7
:1026C0000B7828B11BB9FFF7FDFE01230B7008BD85
:1026D000002BFCD00870BDE80840FFF709BF00BF21
:1026E000EE3302200244074BD2B210B5904200D123
:1026F00010BD441C00B253F8200041F8040BE0B2B6
:10270000F4E700BF502800400F4B30B51C6F240485
:1027100007D41C6F44F400741C671C6F44F400441D
:102720001C670A4C02442368D2B243F480732360CE
:10273000074B904200D130BD441C51F8045B00B2FD
:1027400043F82050E0B2F4E7003802400070004047
:102750005028004007B5012201A90020FFF7C2FF61
:10276000019803B05DF804FB13B50446FFF7F2FFD0
:10277000A04205D0012201A900200194FFF7C4FF67
:1027800002B010BD0144BFF34F8F064B884204D303
:10279000BFF34F8FBFF36F8F7047C3F85C022030D9
:1027A000F4E700BF00ED00E0034B1A681AB9034AD2
:1027B000D2F874281A607047243402200030024096
:1027C00008B5FFF7F1FF024B1868C0F3407008BD71
:1027D0002434022070B5BFF34F8FBFF36F8F1A4AB6
:1027E0000021C2F85012BFF34F8FBFF36F8F5369B0
:1027F00043F400335361BFF34F8FBFF36F8FC2F8C1
:102800008410BFF34F8FD2F8803043F6E074C3F3E7
:10281000C900C3F34E335B0103EA0406014646EAEE
:1028200081750139C2F86052F9D2203B13F1200FB3
:10283000F2D1BFF34F8F536943F480335361BFF339
:102840004F8FBFF36F8F70BD00ED00E0FEE700001B
:10285000214B2248224A70B5904237D3214BC11EEA
:10286000DA1C121A22F003028B4238BF0022002128
:10287000FEF7AAFA1C4A0023C2F88430BFF34F8F38
:10288000D2F8803043F6E074C3F3C900C3F34E338B
:102890005B0103EA0406014646EA81750139C2F884
:1028A0006C52F9D2203B13F1200FF2D1BFF34F8FBE
:1028B000BFF36F8FBFF34F8FBFF36F8F0023C2F84B
:1028C0005032BFF34F8FBFF36F8F70BD53F8041BAF
:1028D00040F8041BC0E700BF7440000838350220F0
:1028E000383502203835022000ED00E070B5D0E91F
:1028F0001B4300224FF0FF359E6804EB4213510149
:10290000D3F80009002805DAD3F8000940F0804028
:10291000C3F80009D3F8000B002805DAD3F8000B40
:1029200040F08040C3F8000B013263189642C3F8B0
:102930000859C3F8085BE0D24FF00113C4F81C3803
:1029400070BD0000890141F02001016103699B060F
:10295000FCD41220FFF7AABA10B5054C2046FEF7AA
:1029600071FF4FF0A043E366024B236710BD00BF29
:1029700028340220C43E000870B503780546012BB8
:1029800050D12A4BC46E98421BD1294B0E214320B3
:102990005A6B42F080025A635A6D42F080025A65C7
:1029A0005A6D5A6942F080025A615A6922F08002D7
:1029B0005A615B6900F034FC1E4BE3601E4BC4F8A7
:1029C00000380023EE6EC4F8003EC02323604FF4AD
:1029D0000413A3633369002BFCDA01230C20336159
:1029E000FFF764FA3369DB07FCD41220FFF75EFAC5
:1029F0003369002BFCDA00262846A660FFF776FF35
:102A00006B68C4F81068DB68C4F81468C4F81C6804
:102A10004BB90A4BA3614FF0FF336361A36843F0E6
:102A20000103A36070BD064BF4E700BF2834022009
:102A3000003802404014004003002002003C30C037
:102A4000083C30C0F8B5C46E054600214FF0006662
:102A50002046FFF777FF296F00234FF001128F68A0
:102A60004FF0FF30C4F83438C4F81C2804EB43128C
:102A700001339F42C2F80069C2F8006BC2F808092E
:102A8000C2F8080BF2D20B68EA6E6B676362102320
:102A90001361166916F01006FBD11220FFF706FA33
:102AA000D4F8003823F4FE63C4F80038A36943F473
:102AB000402343F01003A3610923C4F81038C4F87D
:102AC00014380A4BEB604FF0C043C4F8103B084B7E
:102AD000C4F8003BC4F81069C4F800396B6F03F107
:102AE000100243F480136A67A362F8BDA03E000899
:102AF00040800010C26E90F86610D2F8003823F4BF
:102B0000FE6343EA0113C2F8003870472DE9F84329
:102B100000EB8103C56E0C468046DA680FFA81F936
:102B20004801166806F00306731E022B05EB4113DD
:102B30004FF0000194BFB604384EC3F8101B4FF09D
:102B4000010104F1100398BF06F1805601FA03F366
:102B5000916998BF06F5004600293AD0578A04F1DA
:102B60005801374349016F50D5F81C180B43002119
:102B7000C5F81C382B180127C3F81019A740536952
:102B8000611E9BB3138A928B9B08012A88BF534313
:102B9000D8F87420981842EA034301F14002214614
:102BA000C8F87400284605EB82025360FFF7CAFE9E
:102BB00008EB8900C3681B8A43EA845348341E43E8
:102BC00064012E51D5F81C381F43C5F81C78BDE8A8
:102BD000F88305EB4917D7F8001B21F40041C7F82B
:102BE000001BD5F81C1821EA0303C0E704F13F03DA
:102BF0000B4A2846214605EB83035A60FFF7A2FEE5
:102C000005EB4910D0F8003923F40043C0F800392F
:102C1000D5F81C3823EA0707D7E700BF008000106B
:102C200000040002026F12684267FFF75FBE0000F7
:102C30005831C36E49015B5813F4004004D013F4BB
:102C4000001F0CBF02200120704700004831C36EF6
:102C500049015B5813F4004004D013F4001F0CBF6B
:102C6000022001207047000000EB8101CB68196A47
:102C70000B6813604B6853607047000000EB8103E2
:102C800030B5DD68AA691368D36019B9402B84BFD9
:102C9000402313606B8A1468C26E1C4402EB41101F
:102CA000013C09B2B4FBF3F46343033323F00303A1
:102CB00043EAC44343F0C043C0F8103B2B6803F021
:102CC0000303012B0ED1D2F8083802EB411013F4A4
:102CD000807FD0F8003B14BF43F0805343F0005393
:102CE000C0F8003B02EB4112D2F8003B43F0044332
:102CF000C2F8003B30BD00002DE9F041244D0446F0
:102D0000EE6E06EB4013D3F8087B3807C3F8087B58
:102D10000AD5D6F81438190706D505EB84032146E1
:102D20002846DB685B689847FA071FD5D6F8143841
:102D3000DB071BD505EB8403D968CCB98B69488ABE
:102D40005A68B2FBF0F600FB16228AB91868DA68F6
:102D500090420DD2121AC3E90024302383F3118864
:102D60000B482146FFF78AFF84F31188BDE8F08104
:102D7000012303FA04F26B8923EA02036B81CB6817
:102D8000002BF3D021460248BDE8F041184700BFB0
:102D90002834022000EB81034A0170B5DD68C36E60
:102DA0006C692668E66056BB1A444FF40020C2F8EE
:102DB00010092A6802F00302012A0AB20ED1D3F8E0
:102DC000080803EB421410F4807FD4F8000914BF04
:102DD00040F0805040F00050C4F8000903EB42126C
:102DE000D2F8000940F00440C2F800090122D3F8EB
:102DF000340802FA01F10143C3F8341870BD19B95F
:102E0000402E84BF4020206020681A442E8A8419F6
:102E1000013CB4FBF6F440EAC44040F00050C6E781
:102E20002DE9F8433B4D04464701EE6E06EB401397
:102E3000D3F8088918F0010FC3F808891AD0D6F81A
:102E40001038DB0716D505EB8003D9684B69186885
:102E5000DA68904230D2121A4FF000091A60C3F8B3
:102E60000490302383F3118821462846FFF792FF10
:102E700089F3118818F0800F1CD0D6F83438012659
:102E8000A640334216D005EB84030134ED6ED3F82F
:102E90000CC0E4B22F44DCF8142005EB0434D2F863
:102EA00000E05168714515D3D5F8343823EA060699
:102EB000C5F83468BDE8F883012303FA04F22B89CE
:102EC00023EA02032B818B68002BD3D021462846AE
:102ED0009847CFE7AEEB0103BCF81000834228BF50
:102EE0000346D7F8180980B2B3EB800FE2D8906898
:102EF000A0F1040959F8048FC4F80080A0EB090878
:102F00009844B8F1040FF5D818440B44906053600E
:102F1000C7E700BF283402202DE9F74FA44CE56E27
:102F20006E69AB691E4016F480586E6107D020466A
:102F3000FEF7F6FC03B0BDE8F04F00F069BC002ED0
:102F400012DAD5F8003E9B0705D0D5F8003E23F0F5
:102F50000303C5F8003ED5F80438954823F0010373
:102F6000C5F80438FEF708FD370505D59048FFF78A
:102F7000BDFC8F48FEF7EEFCB0040CD5D5F8083840
:102F800013F0060FEB6823F470530CBF43F4105397
:102F900043F4A053EB6031071BD56368DB681BB9B2
:102FA000AB6923F00803AB612378052B0CD1D5F86E
:102FB000003E9A0705D0D5F8003E23F00303C5F87C
:102FC000003E7B48FEF7D8FC6368DB680BB17848AD
:102FD0009847F30200F18980B70227D5D4F86C90A6
:102FE00000274FF0010ADFF8C8B109EB4712D2F809
:102FF000003B03F44023B3F5802F11D1D2F8003BFE
:10300000002B0DDA62890AFA07F322EA03036381CF
:1030100004EB8703DB68DB6813B1394658469847F1
:103020000137236FFFB29B689F42DED9F00617D5A8
:10303000E76E3A6AC2F30A1002F00F0302F4F012CC
:10304000B2F5802F00F09880B2F5402F08D104EB44
:103050008303002207F58057DB681B6A90427ED10C
:103060003303D5F818481DD5E70302D50020FFF734
:1030700043FEA50302D50120FFF73EFE600302D503
:103080000220FFF739FE210302D50320FFF734FEAB
:10309000E20202D50420FFF72FFEA30202D505208D
:1030A000FFF72AFE77037FF545AFE60702D500203C
:1030B000FFF7B6FEA50702D50120FFF7B1FE6007B6
:1030C00002D50220FFF7ACFE210702D50320FFF74F
:1030D000A7FEE20602D50420FFF7A2FEA3067FF5B5
:1030E00029AF0520FFF79CFE24E7E36E00274FF091
:1030F0000109DFF8BCA00193236F5FFA87FB9B688F
:103100009B453FF669AF019B03EB4B13D3F80019C6
:1031100001F44021B1F5802F1FD1D3F80019002907
:103120001BDAD3F8001941F09041C3F80019D3F825
:1031300000190029FBDB5946E06EFFF703FC2189EB
:1031400009FA0BF321EA0303238104EB8B03DB6809
:103150009B6813B15946504698470137CCE7910711
:1031600001D1D7F80080072A02F101029CBF03F8C1
:10317000018B4FEA182871E7023307F5805704EBFB
:1031800083025268D2F818C0DCF80820DCE9001C81
:10319000A1EB0C0C002188420CD104EB8304636882
:1031A0009B699A6802449A605A6802445A6057E7D9
:1031B0002834022011F0030F01D1D7F800808C458C
:1031C00001F1010184BF02F8018B4FEA1828E2E700
:1031D000C36E03EB4111D1F8003B43F40013C1F877
:1031E000003B7047C36E03EB4111D1F8003943F443
:1031F0000013C1F800397047C36E03EB4111D1F8D9
:10320000003B23F40013C1F8003B7047C36E03EB8F
:103210004111D1F8003923F40013C1F80039704787
:10322000090100F16043012203F56143C9B283F84B
:10323000001300F01F039A4043099B0003F1604311
:1032400003F56143C3F880211A60704730B5043339
:10325000039C0172002104FB0325C160C0E90653F1
:10326000049B0363059BC0E90000C0E90422C0E998
:103270000842C0E90A11436330BD00000022416AE0
:10328000C260C0E90411C0E90A226FF00101FEF733
:103290007DBE0000D0E90432934201D1C2680AB970
:1032A000181D704700207047036919600021C2682B
:1032B0000132C260C269134482699342036124BF30
:1032C000436A0361FEF756BE38B504460D46E3680F
:1032D0003BB162690020131D1268A3621344E362CC
:1032E00007E0237A33B929462046FEF733FE00284B
:1032F000EDDA38BD6FF00100FBE70000C368C2697A
:10330000013BC3604369134482699342436124BF14
:10331000436A436100238362036B03B1184770471C
:1033200070B53023044683F31188866A3EB9FFF7EF
:10333000CBFF054618B186F31188284670BDA36AF5
:10334000E26A13F8015B9342A36202D32046FFF7BF
:10335000D5FF002383F31188EFE700002DE9F84F34
:1033600004460E46174698464FF0300989F31188F7
:103370000025AA46D4F828B0BBF1000F09D1414678
:103380002046FFF7A1FF20B18BF311882846BDE846
:10339000F88FD4E90A12A7EB050B521A934528BF00
:1033A0009346BBF1400F1BD9334601F1400251F85F
:1033B000040B914243F8040BF9D1A36A403640351F
:1033C0004033A362D4E90A239A4202D32046FFF78E
:1033D00095FF8AF31188BD42D8D289F31188C9E7D5
:1033E00030465A46FDF7CAFCA36A5E445D445B441E
:1033F000A362E7E710B5029C0433017203FB0421CA
:10340000C460C0E906130023C0E90A33039B0363C9
:10341000049BC0E90000C0E90422C0E908424363FC
:1034200010BD0000026A6FF00101C260426AC0E98B
:1034300004220022C0E90A22FEF7A8BDD0E9042335
:103440009A4201D1C26822B9184650F8043B0B6079
:10345000704700231846FAE7C3680021C2690133A8
:10346000C3604369134482699342436124BF436A42
:103470004361FEF77FBD000038B504460D46E368A2
:103480003BB1236900201A1DA262E2691344E36282
:1034900007E0237A33B929462046FEF75BFD002872
:1034A000EDDA38BD6FF00100FBE700000369196039
:1034B000C268013AC260C2691344826993420361DF
:1034C00024BF436A036100238362036B03B118477F
:1034D0007047000070B530230D460446114683F353
:1034E0001188866A2EB9FFF7C7FF10B186F31188DD
:1034F00070BDA36A1D70A36AE26A01339342A3629E
:1035000004D3E16920460439FFF7D0FF002080F39F
:103510001188EDE72DE9F84F04460D46904699468F
:103520004FF0300A8AF311880026B346A76A4FB9D4
:1035300049462046FFF7A0FF20B187F311883046A7
:10354000BDE8F88FD4E90A073A1AA8EB06079742B4
:1035500028BF1746402F1BD905F1400355F8042B0F
:103560009D4240F8042BF9D1A36A40364033A36250
:10357000D4E90A239A4204D3E16920460439FFF7CB
:1035800095FF8BF311884645D9D28AF31188CDE790
:1035900029463A46FDF7F2FBA36A3D443E443B44CC
:1035A000A362E5E7D0E904239A4217D1C3689BB12F
:1035B000836A8BB1043B9B1A0ED01360C368013B36
:1035C000C360C3691A4483699A42026124BF436A93
:1035D0000361002383620123184670470023FBE741
:1035E00000F040B94FF08043586A70474FF0804375
:1035F000002258631A610222DA6070474FF080435C
:103600000022DA60704700004FF080435863704733
:10361000FEE7000070B51B4B0025044686B05860DD
:103620000E468562016300F0CBF804F11003A5603B
:10363000E562C4E904334FF0FF33C4E90044C4E950
:103640000635FFF7CFFF2B46024604F13401204632
:10365000C4E9082380230C4A2565FEF731FC0123C9
:103660000A4AE06000920375684672680192B26887
:10367000CDE90223064BCDE90435FEF749FC06B03F
:1036800070BD00BFB0280220D03E0008D53E000823
:1036900011360008024AD36A1843D062704700BF4F
:1036A000482602204B6843608B688360CB68C36008
:1036B0000B6943614B6903628B6943620B6803606A
:1036C0007047000008B52C4B40F2FF712B481A6977
:1036D0000A431A611A6922F4FF6222F007021A6192
:1036E0001A691A6B0A431A631A6D0A431A65244A47
:1036F0001B6D1146FFF7D6FF00F5806002F11C013B
:10370000FFF7D0FF00F5806002F13801FFF7CAFF34
:1037100000F5806002F15401FFF7C4FF00F58060FE
:1037200002F17001FFF7BEFF00F5806002F18C012D
:10373000FFF7B8FF00F5806002F1A801FFF7B2FFC4
:1037400000F5806002F1C401FFF7ACFF00F5806076
:1037500002F1E001FFF7A6FF00F5806002F1FC0135
:10376000FFF7A0FF02F58C7100F58060FFF79AFF6C
:10377000BDE8084000F0ECB800380240000002400C
:10378000DC3E000808B500F065FAFEF777FBFFF7AE
:103790000BF8BDE80840FEF7E5BD000070470000EB
:1037A000EFF30983054968334A6B22F001024A634B
:1037B00083F30988002383F31188704700EF00E04A
:1037C000302080F3118862B60D4B0E4AD96821F47F
:1037D000E0610904090C0A430B49DA60D3F8FC20C4
:1037E00042F08072C3F8FC20084AC2F8B01F11688A
:1037F00041F0010111602022DA7783F8220070473E
:1038000000ED00E00003FA0555CEACC5001000E065
:10381000302310B583F311880E4B5B6813F40063FB
:1038200014D0F1EE103AEFF309844FF08073683C46
:10383000E361094BDB6B236684F30988FEF7FEFA2C
:1038400010B1064BA36110BD054BFBE783F3118854
:10385000F9E700BF00ED00E000EF00E04F030008D3
:10386000520300080F4B1A6C42F001021A641A6EE0
:1038700042F001021A660C4A1B6E936843F0010382
:1038800093604FF080436B229A624FF0FF32DA620E
:1038900000229A615A63DA605A6001225A611A6002
:1038A000704700BF00380240002004E04FF0804223
:1038B00008B51169D3680B40D9B29B076FEA0101C3
:1038C000116107D5302383F31188FEF7EDFA002349
:1038D00083F3118808BD00001B4B4FF0FF3000211F
:1038E0001A696FEA42526FEA52521A611A69C2F3B8
:1038F0000A021A611A695A6958615A6959615A6902
:103900001A6A62F080521A621A6A02F080521A62CF
:103910001A6A5A6A58625A6A59625A6A0B4A106895
:1039200040F480701060186F00F44070B0F5007FB4
:1039300003D04FF4803018671967536823F400737D
:10394000536000F05FB900BF0038024000700040D3
:10395000364B4FF44041364A1A64364A11601A68B1
:1039600042F001021A601A689207FCD59A6822F0A8
:1039700003029A602D4B9A6812F00C02FBD1196871
:1039800001F0F90119609A601A6842F480321A60F5
:103990001A689003FCD55A6F42F001025A67234B14
:1039A0005A6F9107FCD5244A5A601A6842F0807217
:1039B0001A60204B5A685204FCD51A6842F48032CF
:1039C0001A605A68D003FCD51A6842F400321A60B3
:1039D000184A53689903FCD5144B1A689201FCD518
:1039E000164A9A6040F20112C3F88C200022C3F8F4
:1039F000902040F20733124A1360136803F00F035C
:103A0000072BFAD1094B9A6842F002029A609A6831
:103A100002F00C02082AFAD15A6C42F480425A642D
:103A20005A6E42F480425A665B6E7047003802401C
:103A30000004001000700040086C400900948838B1
:103A4000003C0240074A08B5536903F00103536183
:103A500023B1054A13680BB150689847BDE8084088
:103A6000FFF7D6BE003C0140B8340220074A08B533
:103A7000536903F00203536123B1054A93680BB104
:103A8000D0689847BDE80840FFF7C2BE003C01403F
:103A9000B8340220074A08B5536903F004035361A0
:103AA00023B1054A13690BB150699847BDE8084036
:103AB000FFF7AEBE003C0140B8340220074A08B50B
:103AC000536903F00803536123B1054A93690BB1AD
:103AD000D0699847BDE80840FFF79ABE003C014016
:103AE000B8340220074A08B5536903F01003536144
:103AF00023B1054A136A0BB1506A9847BDE80840E4
:103B0000FFF786BE003C0140B8340220164B10B5CA
:103B10005C6904F478725A61A30604D5134A936A67
:103B20000BB1D06A9847600604D5104A136B0BB1ED
:103B3000506B9847210604D50C4A936B0BB1D06BA0
:103B40009847E20504D5094A136C0BB1506C9847AD
:103B5000A30504D5054A936C0BB1D06C9847BDE81A
:103B60001040FFF755BE00BF003C0140B8340220B2
:103B7000194B10B55C6904F47C425A61620504D5A6
:103B8000164A136D0BB1506D9847230504D5134A9F
:103B9000936D0BB1D06D9847E00404D50F4A136EB6
:103BA0000BB1506E9847A10404D50C4A936E0BB12B
:103BB000D06E9847620404D5084A136F0BB1506F5A
:103BC0009847230404D5054A936F0BB1D06F9847EB
:103BD000BDE81040FFF71CBE003C0140B834022095
:103BE00008B50348FDF742FABDE80840FFF710BEEC
:103BF000D823022008B5FFF759FEBDE80840FFF7BB
:103C000007BE0000062108B50846FFF709FB06219C
:103C10000720FFF705FB06210820FFF701FB06211F
:103C20000920FFF7FDFA06210A20FFF7F9FA06211D
:103C30001720FFF7F5FA06212820FFF7F1FA0721F0
:103C40001C20FFF7EDFA0C215220BDE80840FFF7D9
:103C5000E7BA000008B5FFF73FFE00F00DF8FDF7EA
:103C60001DFCFDF7EDFDFDF7C5FCFFF797FDBDE879
:103C70000840FFF7B5BC00000023054A1946013390
:103C8000102BC2E9001102F10802F8D1704700BF01
:103C9000B8340220034611F8012B03F8012B002A47
:103CA000F9D1704753544D3332463F3F3F3F3F3F7A
:103CB0000053544D333246375B347C355D780053C6
:103CC000544D333246375B367C375D780000000058
:103CD000009600000000000000000000000000004E
:103CE0000000000000000000000000005D1400085B
:103CF0004914000885140008711400087D14000898
:103D000069140008551400084114000891140008B3
:103D100000000000711500085D15000899150008E5
:103D200085150008911500087D1500086915000823
:103D300055150008A515000800000000010000004E
:103D40000000000063300000443D0008A02602206F
:103D5000B02802204172647550696C6F740025426E
:103D60004F415244252D424C002553455249414C68
:103D70002500000002000000000000008D17000870
:103D8000F917000840004000603102207031022025
:103D9000020000000000000003000000000000001E
:103DA0003D180008000000001000000080310220D3
:103DB0000000000001000000000000002834022084
:103DC000010102000123000811220008AD220008B1
:103DD0009122000843000000DC3D00080902430076
:103DE000020100C0320904000001020201000524A2
:103DF000001001052401000104240202052406002C
:103E000001070582030800FF09040100020A0000FF
:103E10000007050102400000070581024000000084
:103E200012000000283E00081201100102000040AC
:103E300009124157000201020301000004030904B2
:103E400025424F41524425004D6174656B4637361B
:103E5000352D53452D626473686F740030313233F1
:103E60003435363738394142434445460000000076
:103E70000080000000800000008000000080000042
:103E80000000020000000400000004000000040024
:103E90000000040000000400000004000000040012
:103EA0000000000091190008491C0008F51C0008DA
:103EB00040004000A0340220A03402200100000095
:103EC000B034022080000000400100000500000026
:103ED0006D61696E0069646C650000000000802AF5
:103EE00000000000AAAAAAAA00000024FFFF000008
:103EF0000000000000A00A00000000010000000017
:103F0000AAAAAAAA00000001FFFF0000000000000A
:103F1000000000000001000000000000AAAAAAAAF8
:103F200000010000FFFF0000000000000000000092
:103F30000040100000000000AAAAAAAA0040000049
:103F4000FFFB0000000000000000000000814200B4
:103F500000000000AAAAAAAA00404100EFFF00004A
:103F600000000080080000000000000000000000C9
:103F7000AAAAAAAA00000000FFFF0000000000009B
:103F8000000000000000000000000000AAAAAAAA89
:103F900000000000FFFF0000000000000000000023
:103FA0000000000000000000AAAAAAAA0000000069
:103FB000FFFF000000000000000000000000000003
:103FC00000000000AAAAAAAA00000000FFFF00004B
:103FD00000000000000000000000000000000000E1
:103FE00000000000000000000000000000000000D1
:103FF00000000000000000000000000000000000C1
:1040000000000000000000000000000000000000B0
:104010008F0000000000000000801E000000000073
:10402000FF000000B8280220D82302200000000072
:10403000A43C000849040000B13C00085104000001
:10404000BF3C000800960000000008009600000039
:1040500000080000040000003C3E000800000000D2
:104060000000000000000000000000000000000050
:04407000000000004C
:00000001FF
